:100000000C943E000C945B000C945B000C945B0021
:100010000C945B000C945B000C945B000C945B00F4
:100020000C945B000C945B000C945B000C945B00E4
:100030000C942A020C9451020C946A020C945B00FA
:100040000C945B000C945B000C94CF010C945B004F
:100050000C9493030C945B000C94EB030C945B00E6
:100060000C94F6020C945B000C948F0B0C945B00C8
:100070000C945B000C945B000C945B0011241FBE7D
:10008000CFEFD0E1DEBFCDBF12E0A0E0B1E0E6E30C
:10009000FAE102C005900D92A031B107D9F714E042
:1000A000A0E1B2E001C01D92AE39B107E1F70E94B4
:1000B00068000C94190D0C9400008FE184B98DEF49
:1000C00087B984E08AB982E088B980EB8BB908955A
:1000D000AF92BF92CF92DF92EF92FF920F931F9356
:1000E000DF93CF93CDB7DEB727970FB6F894DEBF77
:1000F0000FBECDBF8FE184B98DEF87B984E08AB997
:1001000082E088B980EB8BB90E94B9010E94F002AD
:1001100010924E0486E480934F0488E0809350044C
:1001200081E0809351040E9433031092100285EB0A
:1001300092E090934902809348028FEE92E0909370
:100140004B0280934A0280E092E090936E0280938B
:100150006D029093700280936F02789480911802E0
:100160008823E1F3109218020E9426050E94780568
:100170000E9417060E944A0380E091E00E947904E1
:100180000E944A03109210025EE2A52E41E4B42EB2
:100190007E010894E11CF11C00E234E6C32ED12C50
:1001A00080911002853089F480912B02813069F4AE
:1001B00080910B0390910C03019790930C03809313
:1001C0000B0380910B0390910C03809127028823ED
:1001D00009F461C020912802243608F023E6822F1A
:1001E0006AE00E94F90C882311F4098302C0805D43
:1001F0008983822F6AE00E94F90C905D9A83AB821A
:1002000080912902805D8C83BD821E820E94F90448
:1002100081E065E00E940105C7010E940D05E091A3
:100220004202F0E0EE0FFF1FEE0FFF1FE059FB4F01
:100230001081812F64E60E94F90C282F812F0E94E3
:10024000F90C392F222311F4098302C0205D298380
:10025000832F6AE00E94F90C805D8A83AB82832F32
:100260000E94F90C905D9C83BD821E8281E060E05B
:100270000E940105C7010E940D05812F90E00E9498
:1002800093040E944A0381E06BE00E9401050E94F2
:10029000FD041092270280912502813041F4809163
:1002A0001002813011F40E94B4081092250280914E
:1002B0001B02813031F410921B020E94D4070E946D
:1002C000CE0680911A02813021F510921A02809197
:1002D00010028530F1F480911302E0914202F0E0C7
:1002E000EE0FFF1FEE0FFF1FE259FB4F808380913F
:1002F0002B02813071F410924102D0920C03C09213
:100300000B030E944A0B83E191E00E9479040E9452
:100310004A0380911802813041F4109218028091B2
:100320001002813011F40E9402098091170281307D
:1003300089F41092170280911002853059F41091BF
:10034000130280911402811719F0812F0E94AF05CA
:100350001093140280911902813009F021CF10927C
:1003600019021ECFF89487E080936E007894089568
:10037000089582E085BD109280008093810084EF13
:1003800091E0909389008093880080ED97E09093AE
:100390008B0080938A0081E080936E0008951F9205
:1003A0000F920FB60F9211248F939F9380912F027B
:1003B0008F5F80932F028150893029F481E08093F0
:1003C0001B0210922F0280910A038F5F80930A0311
:1003D00080910A038136B9F591E090931902109249
:1003E0000A0380912E028F5F80932E0280912E024D
:1003F000853021F410922E0290931A0280912C02E3
:100400008F5F80932C0280912C02843639F41092F5
:100410002C0281E0809316028093180280912C02B6
:10042000823319F481E08093180280912D028F5F4E
:1004300080932D0280912D028A3029F410922D0292
:1004400081E0809317029F918F910F900FBE0F90C4
:100450001F9018951F920F920FB60F9211242F9391
:100460003F934F935F936F937F938F939F93AF933C
:10047000BF93EF93FF93E0914802F09149020995F1
:10048000FF91EF91BF91AF919F918F917F916F916C
:100490005F914F913F912F910F900FBE0F901F9042
:1004A00018951F920F920FB60F9211248F939F935E
:1004B0002C98419891E09093240280911102883009
:1004C00011F4909325029F918F910F900FBE0F9082
:1004D0001F9018951F920F920FB60F9211248F93B1
:1004E0009F93EF93FF932C9A1092850010928400B3
:1004F000E0911102F0E0EE0FFF1FE35FFC4F8081FF
:10050000918190938B0080938A00809111028230B8
:1005100089F0833028F4882341F0813091F407C0BA
:10052000833059F0843069F40BC02B9A0AC02B98A1
:100530002A9A07C02A98299A04C02998289A01C0A3
:100540002898809111028F5F80931102809111028F
:10055000893010F010921102FF91EF919F918F91CD
:100560000F900FBE0F901F901895809130029091C0
:100570003102892BA1F4809186009091870090939D
:10058000370280933602809181008F7B80938100B7
:1005900081E090E090933102809330020895809141
:1005A00086009091870090933502809334022091C9
:1005B000810020642093810020913602309137021F
:1005C000821B930B9093330280933202109231027C
:1005D000109230029093B7038093B6030895089564
:1005E00010927C008FEE80937A0008951F920F92F4
:1005F0000FB60F9211248F939F93EF93FF93109256
:100600007A00E0911502F0E08091780090917900F5
:10061000EE0FFF1FEF59FD4F9183808380911502EC
:100620008F5F8093150280911502873010F0109231
:1006300015028091150280937C008FEE80937A00E2
:100640008091610290916202969587959695879523
:1006500080931302FF91EF919F918F910F900FBEA6
:100660000F901F90189580E18093C4001092C500F0
:1006700088E18093C10086E08093C20082EC809381
:10068000C0000895982F8091C00085FFFCCF909303
:10069000C6000895909178018091C00085FFFCCF3D
:1006A0009093C600909179018091C00085FFFCCFA6
:1006B0009093C600089527E030E061E070E0482F95
:1006C00050E0F0E3E1E3CB01022E02C0880F991F56
:1006D0000A94E2F784239523181619063CF48091B6
:1006E000C00085FFFCCFE093C60006C08091C0002B
:1006F00085FFFCCFF093C600215030408FEF2F3F95
:10070000380709F7909178018091C00085FFFCCFF0
:100710009093C600909179018091C00085FFFCCF35
:100720009093C60008951F920F920FB60F92112456
:100730008F939F93EF93FF939091C60090936304E0
:100740009D3099F480913902813079F41092390208
:1007500080932A02E091B503F0E0E15EFC4F9083C4
:100760008091B503809338022DC08091390288238F
:1007700019F0813039F514C0933241F480912A0286
:10078000882321F481E0809339025F9A1092B503A7
:100790008091B503E82FF0E0E15EFC4F90830CC040
:1007A000E091B503F0E0E15EFC4F90838091B503EA
:1007B000853930F48091B5038F5F8093B50302C013
:1007C00010923902FF91EF919F918F910F900FBE80
:1007D0000F901F9018951F920F920FB60F92112431
:1007E0002F933F934F935F936F937F938F939F9339
:1007F000AF93BF93EF93FF9380911002843021F564
:1008000080917A018823E1F480913A0290913B0231
:10081000019690933B0280933A02FC01E854FC4F0E
:10082000E081ED3019F08639910539F410923B02E0
:1008300010923A0281E080937A01E093C60004C0EE
:1008400010923B0210923A0280911002833009F01C
:100850003FC080912602813099F08230F9F08823E0
:10086000B9F51092C5008AE08093C4001092C600CA
:100870000E9427080E94420881E08093260228C037
:100880001092C5008093C4001092C60082E080934D
:10089000260210927602109275021AC082E48A959E
:1008A000F1F78091750290917602FC01E557FD4FBA
:1008B00020812093C6000196909376028093750262
:1008C0008091750290917602C29711F410922602DF
:1008D000FF91EF91BF91AF919F918F917F916F9118
:1008E0005F914F913F912F910F900FBE0F901F90EE
:1008F0001895AC01DC010D900020E9F71197A81BB9
:10090000B90B20E030E0FA01E20FF31FE0818091A3
:10091000C00085FFFCCFE093C6002F5F3F4FA217BA
:10092000B30788F708950F931F93DF93CF93CDB745
:10093000DEB764970FB6F894DEBF0FBECDBF8E0151
:100940000F5F1F4FB8014AE050E00E94C80CC80179
:100950000E94790464960FB6F894DEBF0FBECDBF37
:10096000CF91DF911F910F91089580FF02C0449AAB
:1009700001C0449881FF02C0459A01C0459882FF9A
:1009800002C0469A01C0469883FF02C0479A089564
:1009900047980895429A80E197E20197F1F74298CB
:1009A0000895FF920F931F93F82E82958F700E94E7
:1009B000B504429A00E117E2C8010197F1F74298A5
:1009C0008F2D0E94B504429AC8010197F1F7429811
:1009D0001F910F91FF900895439A0E94D1040895AA
:1009E00043980E94D104439A089581E00E94F00444
:1009F00008958CE00E94F00408958DE00E94F004B8
:100A00000895882319F4862F805804C0813011F48A
:100A1000862F80540E94F00408950F931F93CF9364
:100A2000DF93FC0101900020E9F731970E2F081B9E
:100A3000EC0110E004C089910E94EC041F5F1017C4
:100A4000D0F3DF91CF911F910F910895EF92FF9214
:100A50000F931F9388EA91E60197F1F7439883E09B
:100A60000E94B504429A00E117E2C8010197F1F72C
:100A7000429880E5E82E83ECF82EC7010197F1F744
:100A800083E00E94B504429AC8010197F1F74298A9
:100A9000C7010197F1F783E00E94B504429AC801AB
:100AA0000197F1F7429882E00E94B504429AC8018A
:100AB0000197F1F74298C7010197F1F788E20E9488
:100AC000F0048EE00E94F00481E00E94F0048BE7C5
:100AD00091E00E940D0581E06AE00E94010580E836
:100AE00091E00E940D051F910F91FF90EF900895E6
:100AF0000E94F50480E063E00E94010585E891E032
:100B00000E940D0581E060E00E94010580E991E00E
:100B10000E940D050E94F9044F99FECF0E94F50432
:100B200008950F931F93DF93CF9300D000D00F92BF
:100B3000CDB7DEB78E010F5F1F4FB8014AE050E01E
:100B40000E94C80CC8010E940D050F900F900F90D5
:100B50000F900F90CF91DF911F910F9108951F93E8
:100B6000182F0E94F90480E067E00E94010581EAE5
:100B700091E00E940D0580E067E00E940105812F51
:100B800090E00E9491050E94FD0480912302813033
:100B900039F0823039F0882349F480E060E004C005
:100BA00080E001C081E06BE00E9401051F91089583
:100BB00080912B02882349F481E080932B026BE023
:100BC0000E94010585EA91E012C010922B02E0918B
:100BD0004202F0E0EE0FFF1FEE0FFF1FE259FB4F46
:100BE000108281E06BE00E9401058BEA91E00E9497
:100BF0000D0581E06BE00E940105089580912B02B4
:100C00008823A1F4109210028AE0809321021092AE
:100C10001D0280E062E00E940105809142028F5C2B
:100C20000E94EC0480E062E00E940105089581E0EA
:100C30008093210210922202109210020E94F50469
:100C400080E060E00E94010581EB91E00E940D05CB
:100C500080E069E00E94010589EB91E00E940D05AA
:100C600081E060E00E94010580EC91E00E940D05AA
:100C700081E069E00E94010588EC91E00E940D0589
:100C80000E94FD0480E060E00E94010510921D02B8
:100C9000089586E0809321020E94F50481E069E0D6
:100CA0000E9401058EEC91E00E940D050E94FD045A
:100CB00081E069E00E94010510921D020E94F90482
:100CC000089585E0809321020E94F50481E069E0A7
:100CD0000E9401058EEC91E00E940D050E94FD042A
:100CE00081E069E00E94010510921D020E94F90452
:100CF0000E94E108089584E0809321020E94F50497
:100D000081E069E00E9401058EEC91E00E940D05F2
:100D10000E94FD0481E069E00E94010510921D021D
:100D20000E94F9040E940408089587E0809321023C
:100D300010922202109214020E94F50480E060E0FA
:100D40000E94010583ED91E00E940D058091420211
:100D50008F5C0E94EC0480E064E00E94010586ED57
:100D600091E00E940D0580E06BE00E9401058EEC91
:100D700091E00E940D0581E06BE00E9401058BEA85
:100D800091E00E940D050E94FD0480E060E00E9459
:100D9000010510921D020E943E0B089580911D02D4
:100DA000882309F48FC0809121028130C1F58091A0
:100DB0001D0218162CF4809122028F5F809322026C
:100DC00080911D0287FF05C080912202815080938F
:100DD00022028091220287FF03C083E080932202D7
:100DE00080912202843014F010922202809122021B
:100DF000813061F082301CF4882331F010C08230E1
:100E000039F0833061F407C080E003C080E004C0A3
:100E100081E060E002C081E069E00E94010580910C
:100E20002102873079F580911D02181624F48091F3
:100E300022028F5F03C080912202815080932202A0
:100E40008091220287FF03C082E08093220280917A
:100E50002202833014F010922202809122028093A9
:100E6000230280912202813039F0823039F08823C8
:100E700049F480E060E004C080E001C081E06BE004
:100E80000E940105809121028A30D1F480911D02D7
:100E900090914202181614F49F5F01C091509093F4
:100EA000420280914202893010F0109242028091F9
:100EB00042028F5C0E94EC0480E062E00E94010527
:100EC00010921D024F9909C080916002813051F447
:100ED000109227011092600205C081E080936002A9
:100EE0008093270180912701882309F05CC08091BD
:100EF0002102853049F1863034F4813061F084304C
:100F000009F04EC01EC0873021F18730FCF08A30D6
:100F100009F046C039C080912202823011F40E944B
:100F20007B0680912202882311F40E946106809141
:100F30002202833011F40E94950681E080932701FC
:100F40002FC00E94180802C00E94FB080E941706CA
:100F500027C080912202882311F40E94FE0580910F
:100F60002202813011F40E94170680912202823001
:100F7000B9F480912B02813021F0809113028B30E3
:100F800078F40E94D8050CC087E08093210210926B
:100F9000220280E060E00E94010585E0809310025B
:100FA00081E08093270108954C9B02C023E001C09B
:100FB00020E04D9B02C081E0282790912601921BE2
:100FC00090FF21C02093260180911C0292708150D5
:100FD000890F80931C0280911E028150890F80939B
:100FE0001E0280911E0282302CF081E080931D024F
:100FF00010921E0280911E028F3F2CF48FEF80937F
:101000001D0210921E02089583E080931002F8944E
:101010001092C5008093C4008EE08093C20088E4E3
:101020008093C10078941092C60010922602089511
:1010300010921002F8941092C50083E08093C400CF
:101040008EE08093C2001092C1007894089520E051
:1010500030E040E012C0F901EE0FFF1FEF59FD4FE5
:10106000808191819695879596958795F901E557A9
:10107000FD4F80832F5F3F4F4F5F463064F34093B7
:10108000640408951F93CF93DF9310926404C7E61E
:10109000D4E013E060C0FF27E7FDF095E557FD4F72
:1010A0008081809365041092660490E067E674E0A6
:1010B0004AE050E00E94C80CFE0101900020E9F7D0
:1010C0003197E756F440E0936C0480916404682FF4
:1010D000772767FD70958430B4F4660F771F660F2D
:1010E000771F80E00E9401058CED91E00E940D05C4
:1010F00080916C04912F981B60916404660F660FB9
:10110000690F80E01DC064507040660F771F660F46
:10111000771F81E00E9401058CED91E00E940D0592
:1011200080916C04612F681B80916404992787FD6E
:1011300090950497880F991F880F991F680F81E079
:101140000E94010587E694E00E940D0580916404E9
:101150008F5F80936404E0916404E6300CF49BCFCD
:10116000DF91CF911F910895F89480E09DE79093CF
:101170001E0380931D0340E050E0DA01AA0FBB1F5D
:10118000FD01EF59FD4F8081918188519C4F880F5F
:10119000991FA35FBC4F11969C938E9380911D0362
:1011A00090911E032D913C91821B930B90931E03F3
:1011B00080931D034F5F5F4F48305105F1F67894DF
:1011C0000895F89481E0809310021092800082E0EC
:1011D0008093810080ED97E0909389008093880050
:1011E00088EB9BE090938B0080938A0086E080934D
:1011F0006F0078940895F8941092100210926F0086
:1012000078940895AF92BF92CF92DF92EF92FF92BF
:101210000F931F93DF93CF9300D000D00F92CDB7E1
:10122000DEB7EE24FF2400E06E010894C11CD11C3F
:1012300073E0A72EC701880F991FFC01E25BFD4FE9
:1012400020813181FC01EF59FD4F80819181281768
:101250003907A9F180819181969587959695879513
:10126000B6014AE050E00E94C80CF601019000204F
:10127000E9F73197BE2EBC1883E08E1568F080E048
:10128000602F0E9401058FED91E00E940D056A2DEF
:101290006B19600F80E00EC0102F105181E0612F9C
:1012A0000E9401058FED91E00E940D056A2D6B19DA
:1012B000610F81E00E940105C6010E940D05F70142
:1012C000EE0FFF1FDF01AF59BD4F8D919C91E25B87
:1012D000FD4F918380830894E11CF11C0C5F083161
:1012E00009F0A8CF0F900F900F900F900F90CF9113
:1012F000DF911F910F91FF90EF90DF90CF90BF9003
:10130000AF90089584E08093100280E18093C40040
:101310001092C50088ED8093C10086E08093C200E2
:1013200082EC8093C00008951092100280E18093B7
:10133000C4001092C5001092C10086E08093C200E4
:1013400082EC8093C0000895DC0120E030E040E0B2
:1013500050E008C0FA01E854FC4F8081280F311D8D
:101360004F5F5F4F4A175B07A8F33F70C90136E034
:10137000969587953A95E1F7835CFD01E854FC4F1B
:10138000808311962F73235CFD01E854FC4F20836A
:10139000A754BC4F8DE08C9310927A018091B803D2
:1013A0008093C6000895CF93DF93EA01B22F93E2B2
:1013B0009093B8036093B9038093BA0363E070E03D
:1013C000A0E04EC0FE01EA0FF11D9081AF5FB15069
:1013D00019F430E040E00FC0FE01EA0FF11D40813A
:1013E000AF5FB15011F430E006C0FE01EA0FF11D0D
:1013F0003081AF5FB150892F86958695835CFB0164
:10140000E854FC4F8083242F22952F70892F90E081
:101410008370907054E0880F991F5A95E1F7282B3C
:10142000235CFB01E754FC4F2083842F90E08F70F6
:101430009070880F991F880F991F232F229526954A
:1014400026952370282B235CFB01E654FC4F208358
:101450003F73335CFB01E554FC4F30836C5F7F4F7F
:10146000BB2309F0AFCFCB010E94A409DF91CF913C
:101470000895DF93CF93CDB7DEB760970FB6F8949A
:10148000DEBF0FBECDBF80917A01882309F458C01A
:1014900060916D046F3F59F0605D81E4AE014F5F74
:1014A0005F4F20E10E94D3098FEF80936D048091FC
:1014B0003C02813061F487E461E048E554E02BE0D0
:1014C0000E94D30910923C0282E080931202809124
:1014D0003D02813061F482E08093120286E561E092
:1014E0004EE454E02AE00E94D30910923D0280911C
:1014F0003E028130E1F482E080931202809140024A
:1015000044E1849FA0011124485D5E4F805D60E04E
:1015100024E10E94D309809140028F5F80934002B2
:101520008150843011F41092400210923E0280915A
:101530003F02813029F482E08093120210923F0230
:1015400060960FB6F894DEBF0FBECDBFCF91DF918E
:1015500008951F93CF93DF93EC0170E0A22FB0E0CA
:10156000119748C0E42FF0E0E15EFC4F30814F5FFF
:10157000E42FF0E0E15EFC4F50814F5FE42FF0E09C
:10158000E15EFC4F10814F5FE42FF0E0E15EFC4F25
:1015900020814F5F842F90E08A179B0774F55D537D
:1015A000FE01E70FF11D852F82958F703D53330F9C
:1015B000330F382B3083613001F1912F9D537F5FC2
:1015C000FE01E70FF11D71505295507F892F8695CE
:1015D0008695582B5083623081F063507E5FFE0108
:1015E000E70FF11D9295990F990F907C2D53922B37
:1015F00090837F5F662309F0B5CFDF91CF911F9174
:101600000895DF93CF9300D000D0CDB7DEB780919F
:1016100021038736C1F0883628F4813641F08336BD
:1016200021F51DC08836B9F08637F9F410C0209135
:101630003802CE01019664E043E00E94A90A898144
:1016400080936D0412C081E080933C020EC081E063
:1016500080933D020AC081E080933E0206C081E093
:1016600080933F0282E08093120210922A020F9030
:101670000F900F900F90CF91DF91089585E08093A8
:1016800010021092B9008AE28093B8000895109277
:101690001002089585EA8093BC00089584E9809340
:1016A000BC0008954CEB50E084E9DA018C93109271
:1016B00041022BEB30E0F90180811092420280E878
:1016C0008C931092BA001082E9EBF0E01082A8EB44
:1016D000B0E01C9285E08093100210828AE28C9325
:1016E00085EADA018C931082F901108285E88C93E7
:1016F00008951092B9008093BB0085E88093BC00E8
:1017000008958093BB0085E88093BC00089585EC24
:101710008093BC00089585E88093BC0008951F92D3
:101720000F920FB60F9211242F933F934F935F9315
:101730006F937F938F939F93AF93BF93EF93FF9399
:1017400082EE91E00E9479040E944A038091410256
:101750008F5F809341028150853009F4ACC08630A0
:1017600090F4823009F443C0833030F48823F1F0E0
:10177000813009F0F5C023C0833009F466C084309D
:1017800009F0EEC06EC0883009F4C0C0893038F46A
:10179000863009F49DC0873009F0E2C0B3C08930BB
:1017A00009F4BAC08A3009F0DBC0CDC01092B9008C
:1017B0008091420290E08996880F991F0CC0E091B9
:1017C0004202F0E0EE0FFF1FEE0FFF1FE259FB4F4A
:1017D00080811092B9008093BB0085E88093BC00A3
:1017E00084E690E090930C0380930B03BBC0809140
:1017F000B9008033F9F480914702882321F4809165
:1018000042028093470280914202E82FF0E0EE0FFF
:10181000FF1FEE0FFF1FE659FB4F9181892F8F7736
:101820008F3711F09F5F918385EF91E00E947904DB
:101830000E944A0384E98093BC0084E690E0909380
:101840000C0380930B0385EA09C080914202880F44
:101850008D5A1092B9008093BB0085E88093BC003C
:1018600081C08091B900E0914202803481F0F0E0C3
:10187000EE0FFF1FEE0FFF1FE259FB4F81818F77A5
:10188000818384E98093BC00109241020DC0F0E096
:10189000EE0FFF1FEE0FFF1FE259FB4F81818068A3
:1018A000818385EC8093BC00809147028093440241
:1018B0001092470257C08091BB00E0914202F0E0D5
:1018C000EE0FFF1FEE0FFF1FE059FB4F8083C5CFC8
:1018D0008091BB00E0914202F0E0EE0FFF1FEE0F9F
:1018E000FF1FE259FB4F838384E98093BC0084E6A9
:1018F00090E090930C0380930B0385EA8093BC00E7
:1019000081E02BC01092B90089E9A5CF8091B90080
:10191000803431F485ECA2CF8091B900803571F02C
:1019200082E092E00E9479048091B9000E945B03FA
:101930000E944A0384E98093BC0012C08091BB00DE
:10194000809328028ACF8091BB008093290284E98A
:101950008093BC001092410282E08093270202C073
:10196000109241028091BC0080688093BC00FF917E
:10197000EF91BF91AF919F918F917F916F915F9107
:101980004F913F912F910F900FBE0F901F90189580
:10199000FB019F01E8944230C4F04532B4F44A3070
:1019A00029F497FB1EF4909581959F4F642F77271C
:1019B0000E94050D805D8A330CF0895D8193CB0117
:1019C0000097A1F716F45DE251931082C9010C94BF
:1019D000E90CDC01FC01672F71917723E1F7329765
:1019E00004C07C916D9370836291AE17BF07C8F3FA
:1019F0000895991B79E004C0991F961708F0961B6B
:101A0000881F7A95C9F780950895AA1BBB1B51E1E1
:101A100007C0AA1FBB1FA617B70710F0A61BB70B5E
:101A2000881F991F5A95A9F780959095BC01CD0103
:061A30000895F894FFCFB9
:101A3600736572766F7465737420562E20302E3758
:101A46002E73006932635F7374617274004B2000F9
:101A5600000000003D0001013D3D3D204D696372DF
:101A66006F636F62746572203D3D3D0046432D53A2
:101A7600696D756C61746F72205620302E312000AE
:101A860020202020204550492D5445414D2020201E
:101A960020202000202020202020776F77696520D5
:101AA60020202020202020000D0A0168756875007E
:101AB600416B6B75004550492D5465737465720012
:101AC6002D2D2D465245452054494245542D2D2D48
:101AD600002020200053746F7020005374617274CC
:101AE6000050504D2D4F75740050504D2D496E00CD
:101AF600444D582D4F757400424C432D5400457883
:101B0600697400413D00533D202030002020002014
:101B1600200054574920566563746F7220726561C0
:101B2600636865640054575352203D3D2030783336
:101B36003000545749204572726F7220203D2000B4
:00000001FF
